:020000000130CD
:10003000758160120097759038117475903811743D
:100040007590381174759038117475900811747525
:1000500090011174759006117475900C117475905F
:100060008011749000A0117F7590C011749000A849
:10007000117F80BFC2B5C2B6C2B71197D2B722797D
:1000800000E993118A09B910F822F590D2B5C2B6E9
:10009000C2B71197D2B7227FFF7EFFDEFEDFFA22C2
:1000A0002031313131313131202020303537312D7F
:0800B00038353935363032389D
:00000001FF
